:060000000A128A11122809
:10000800FE00030E83120313A8000408A9000A08BF
:10001800AA007F08AB000A128A11292B0A128A1536
:10002800A12A000000008312031362088316031339
:10003800CE0083120313610883160313CD008312C5
:100048000313600883160313CC00831203135F089D
:1000580083160313CB000A128A155F270A128A1126
:100068000A128A151A240A128A11831203136208C3
:10007800CA006108C9006008C8005F08C7000A30E4
:10008800CB000030CC00BF300A128A1567230A1251
:100098008A11203083120313AC008030AD00033086
:1000A800AE000030AF00BC300A128A152F230A12A6
:1000B8008A11831203136208803AFF000030803AE5
:1000C8007F02031D712800306102031D7128003072
:1000D8006002031D71280A305F020318742875280E
:1000E8009A28BF30AC000030AD000130AE000030BF
:1000F800AF00BB300A128A152F230A128A111B304F
:1001080083120313AC008030AD000430AE00003021
:10011800AF00B7300A128A152F230A128A11083045
:1001280083160313A9000030AA00FD2A831262086F
:10013800803AFF000030803A7F02031DAD2800306E
:100148006102031DAD2800306002031DAD280A308E
:100158005F02031CB028B128EC286208803AFF002F
:100168000030803A7F02031DC32800306102031D5E
:10017800C32800306002031DC32864305F020318DF
:10018800C628C728EC28BF30AC000030AD000230CC
:10019800AE000030AF00BA300A128A152F230A12B7
:1001A8008A11243083120313AC008030AD00033071
:1001B800AE000030AF00B7300A128A152F230A129A
:1001C8008A11083083160313A9000030AA00FD2AFB
:1001D80083126208803AFF000030803A7F02031DD4
:1001E800FF2800306102031DFF2800306002031D54
:1001F800FF2864305F02031C022903293E29620894
:10020800803AFF000030803A7F02031D1529003034
:100218006102031D152903306002031D1529E8300A
:100228005F020318182919293E29BF30AC00003095
:10023800AD000330AE000030AF00B9300A128A15A5
:100248002F230A128A11283083120313AC0080303E
:10025800AD000230AE000030AF00B7300A128A1588
:100268002F230A128A11083083160313A9000030BD
:10027800AA00FD2A83126208803AFF000030803A03
:100288007F02031D512900306102031D51290330EB
:100298006002031D5129E8305F02031C54295529C7
:1002A8008E296208803AFF000030803A7F02031DE1
:1002B800672900306102031D672927306002031D8A
:1002C800672910305F0203186A296B298E29C0300C
:1002D800AC000030AD000330AE000030AF00B930E4
:1002E8000A128A152F230A128A112E308312031339
:1002F800D800580883160313B8003F088312031365
:10030800D800580883160313B7000830A900003036
:10031800AA00FD2A83126208803AFF000030803A62
:100328007F02031DA12900306102031DA129273086
:100338006002031DA12910305F02031CA429A5290E
:10034800E8296208803AFF000030803A7F02031DE6
:10035800B72901306102031DB72986306002031DE9
:10036800B729A0305F020318BA29BB29E829C13090
:10037800AC000030AD000330AE000030AF00B93043
:100388000A128A152F230A128A112E308312031398
:10039800D800580883160313B800BF30831203131C
:1003A800AC000030AD000230AE000030AF00B63017
:1003B8000A128A152F230A128A1109308316031389
:1003C800A9000030AA00FD2A83126208803AFF00C3
:1003D8000030803A7F02031DFB2901306102031DB2
:1003E800FB2986306002031DFB29A0305F02031C35
:1003F800FE29FF29422A6208803AFF000030803A2D
:100408007F02031D112A0F306102031D112A423099
:100418006002031D112A40305F020318142A152AAE
:10042800422AC230AC000030AD000330AE000030CC
:10043800AF00B9300A128A152F230A128A112E30FA
:1004480083120313D800580883160313B800BF306B
:1004580083120313AC000030AD000330AE0000304F
:10046800AF00B5300A128A152F230A128A110A30F2
:1004780083160313A9000030AA00FD2A831262081C
:10048800803AFF000030803A7F02031D552A0F3062
:100498006102031D552A42306002031D552A40306F
:1004A8005F02031C582A592A9C2A6208803AFF00D6
:1004B8000030803A7F02031D6B2A98306102031DC9
:1004C8006B2A96306002031D6B2A80305F02031886
:1004D8006E2A6F2A9C2AC330AC000030AD0003306E
:1004E800AE000030AF00B9300A128A152F230A1265
:1004F8008A112E3083120313D80058088316031369
:10050800B800BF3083120313AC000030AD000430D4
:10051800AE000030AF00B4300A128A152F230A1239
:100528008A110B3083160313A9000030AA00FD2A94
:1005380083126208803AFF000030803A7F02031D70
:10054800AF2A98306102031DAF2A96306002031D5E
:10055800AF2A80305F02031CB22AB32AFD2A620840
:10056800803AFF000530803A7F02031DC52AF53026
:100578006102031DC52AE1306002031DC52A00304F
:100588005F020318C82AC92AFD2AC430AC0000300B
:10059800AD000330AE000030AF00B9300A128A1542
:1005A8002F230A128A112E3083120313D8005808F9
:1005B80083160313B800BF3083120313AC00003056
:1005C800AD000530AE000030AF00B3300A128A1516
:1005D8002F230A128A110C3083160313A900003046
:1005E800AA00FD2AFD2AFD2AFD2AFD2AFD2AFD2A48
:1005F800FD2A0A128A1512220A128A1104300A12D6
:100608008A15FF220A128A11103083120313D800A8
:10061800D80B0C2B00000D300A128A1529220A1259
:100628008A11AF3083120313D8005808B00083161C
:10063800031329080A128A159F230A128A110A121B
:100648008A118F260A128A110800000000008312FE
:1006580003130C10D8308F00F0308E00051A352B9C
:10066800362B142CFD305C02E83003195B020318AA
:100678003E2B3F2B172C0130DB070318DC0A003018
:10068800DC0702305B065C04031D4B2B4C2BA02BB4
:100698005F0883160313580783120313A000003062
:1006A800031801306007A2010318A20A8316031376
:1006B800590783120313A1000318A20A610822072D
:1006C800A3010318A30A831603135A0783120313FB
:1006D800A2000318A30A62082307831603135B0703
:1006E80083120313A3002308E2002208E100210873
:1006F800E0002008DF006208803AFF000430803AFA
:100708007F02031D912B2C306102031D912B1D309C
:100718006002031D912B81305F02031C942B952BE3
:100728009E2B0430E2002C30E1001D30E0008030C8
:10073800DF009E2B5D14A02B3230F0000030F1005A
:100748005C08F301F3075B08F201F2070A128A1545
:10075800D7230A128A1171087004031DB42BB52B14
:10076800172C831603135B08F3005A08F200590884
:10077800F1005808F0000030F7000030F6000030B3
:10078800F5000530F4000A128A155D240A128A1150
:100798007008831203135F07A000003003180130AC
:1007A8007107A2010318A20A6007A1000318A20A90
:1007B80072082207A3010318A30A6107A2000318FD
:1007C800A30A730823076207A3002308E20022088C
:1007D800E1002108E0002008DF006208803AFF00FD
:1007E8000430803A7F02031D032C2C306102031D64
:1007F800032C1D306002031D032C81305F02031C93
:10080800062C072C102C0430E2002C30E1001D309F
:10081800E0008030DF00102C5D14172C172C172CEB
:10082800DB01DC01172C8312031307191C2C1D2C68
:10083800192DFD305A02E830031959020318252CE6
:10084800262C1C2D0130D9070318DA0A0030DA07E4
:10085800023059065A04031D322C332C952C5F089C
:10086800A0006008A1006108A2006208A300831626
:100878000313580983120313A40083160313590999
:1008880083120313A500831603135A098312031353
:10089800A600831603135B0983120313A700A40A97
:1008A8000319A50A0319A60A0319A70A2408A00709
:1008B80025080318250F612C622CA10726080318A8
:1008C800260F672C682CA20727080318270AA307F6
:1008D8002308E2002208E1002108E0002008DF00E8
:1008E8006208803AFF000030803A7F02031D862CA0
:1008F80000306102031D862C00306002031D862C27
:1009080001305F020318892C8A2C932C0030E200F6
:100918000030E1000030E0000130DF00932C5D146E
:10092800952C3230F0000030F1005A08F301F3073B
:100938005908F201F2070A128A15D7230A128A11F6
:1009480071087004031DA92CAA2C1C2D83120313F3
:100958005F08A0006008A1006108A2006208A30067
:10096800831603135B08F3005A08F2005908F100D4
:100978005808F0000030F7000030F6000030F500AD
:100988000530F4000A128A155D240A128A117009CA
:1009980083120313A4007109A5007209A600730944
:1009A800A700A40A0319A50A0319A60A0319A70A86
:1009B8002408A00725080318250FE32CE42CA10719
:1009C80026080318260FE92CEA2CA2072708031883
:1009D800270AA3072308E2002208E1002108E00013
:1009E8002008DF006208803AFF000030803A7F026A
:1009F800031D082D00306102031D082D0030600220
:100A0800031D082D01305F0203180B2D0C2D152D29
:100A18000030E2000030E1000030E0000130DF008B
:100A2800152D5D141C2D1C2D1C2DD901DA011C2D32
:100A380083120313071A212D222D672DFD308316EB
:100A480003132E02E83003192D0203182C2D2D2D27
:100A58006C2D0130AD070318AE0A0030AE07023026
:100A68002D062E04031D392D3A2D442D8312031310
:100A78006308013E0739A0002008E300DD14442D77
:100A88003230F0000030F100831603132E08F30112
:100A9800F3072D08F201F2070A128A15D7230A1262
:100AA8008A1171087004031D5A2D5B2D6C2D831259
:100AB80003136308013E0739A0002008E300DD1492
:100AC8006C2D6C2D6C2D83160313AD01AE016C2DAE
:100AD800831203132B08FF002A088A0029088400C0
:100AE800280E8300FE0E7E0E0900831203133B08B6
:100AF800C3003C08C4003D08C5003E08C6000310FA
:100B0800450D460DC7004708C800C808031D8D2DB0
:100B18008E2D982D0030BE000030BD000030BC0086
:100B28000030BB008E2E8E2E3F08C3004008C40044
:100B38004108C5004208C6000310450D460DC70010
:100B48004708CE00CE08031DAA2DAB2DB52D0030C9
:100B5800BE000030BD000030BC000030BB008E2E4F
:100B68008E2E4E087B3EC3004308C8073B08C300CF
:100B78003C08C4003D08C5003E08C60018300310F4
:100B8800C60CC50CC40CC30CFF3E031DC32D430883
:100B9800C7004708CE003F08C3004008C40041080A
:100BA800C5004208C60018300310C60CC50CC40C9A
:100BB800C30CFF3E031DD82D4308C7004708CE06C7
:100BC8008030C3004308CE05BD17C117FF30BF05ED
:100BD800FF30C005FF30C1050030C2050030CC0031
:100BE8000030CB000030CA000030C9000730C30015
:100BF8004308CD00FF2D3B1C022E032E1B2E3F0861
:100C0800C907400803110318013E03190C2ECA072F
:100C1800410803110318013E0319132ECB0742089C
:100C280003110318013E03191A2ECC071B2E01309D
:100C38000310BE0CBD0CBC0CBB0CFF3E031D1C2ED0
:100C48000130C3000310BF0DC00DC10DC20DC30B91
:100C5800262E0130CD02031D322E332EFF2D342EC9
:100C68001130C3004308CD00392E3B1C3C2E3D2ECD
:100C7800552E3F08C907400803110318013E031900
:100C8800462ECA07410803110318013E03194D2EC9
:100C9800CB07420803110318013E0319542ECC0751
:100CA800552E01300310BE0CBD0CBC0CBB0CFF3E16
:100CB800031D562E01300310CC0CCB0CCA0CC90CEA
:100CC800FF3E031D5F2E0130CD02031D6C2E6D2EDD
:100CD800392E6E2E4C08AF004B08AE004A08AD0006
:100CE8004908AC004808C3004308B0004E08C400D7
:100CF8004408B1000A128A1535260A128A1183128D
:100D080003132F08BE002E08BD002D08BC002C08B8
:100D1800BB008E2E0800000000002B2F0030831629
:100D28000313DB000030DA000030D9000130D800AE
:100D38000A300A128A1529220A128A11472F00300E
:100D480083160313DB000030DA000030D9000A30C4
:100D5800D80009300A128A1529220A128A11472F47
:100D6800003083160313DB000030DA000030D900AE
:100D78006430D80008300A128A1529220A128A110A
:100D8800472F003083160313DB000030DA000330EE
:100D9800D900E830D80006300A128A1529220A122A
:100DA8008A11472F003083160313DB000030DA0066
:100DB8002730D9001030D80005300A128A152922A8
:100DC8000A128A11472F003083160313DB00013003
:100DD800DA008630D900A030D80004300A128A150B
:100DE80029220A128A11472F003083160313DB00C9
:100DF8000F30DA004230D9004030D80003300A12F0
:100E08008A1529220A128A11472F003083160313E4
:100E1800DB009830DA009630D9008030D8000230F4
:100E28000A128A1529220A128A11472F00308316BE
:100E38000313DB000030DA000330D900E830D800B3
:100E480006300A128A1529220A128A11472F83129C
:100E580003136308003A0319922E013A0319A32ECB
:100E6800033A0319B42E013A0319C52E073A031998
:100E7800D62E013A0319E72E033A0319F82E013A40
:100E88000319092F1A2F0800831203134F08D300E0
:100E98005008D4005108D5005208D6000310550D4B
:100EA800560DD700570883160313CA00CA08031D36
:100EB8005E2F5F2F6B2F003083120313D200003098
:100EC800D1000030D0000030CF00FC2FFC2F83125F
:100ED8004F08D3005008D4005108D5005208D60056
:100EE8001F300310D60CD50CD40CD30CFF3E031DB9
:100EF800752F5308D700570883160313C9008312A8
:100F08000313D117FF30CF05FF30D005FF30D105CF
:100F18000030D205963083160313CA02CA1F952FD4
:100F2800962FC02F4A08803A973E03189C2F9D2F72
:100F3800AA2F003083120313D2000030D1000030F2
:100F4800D0000030CF00FC2FFC2FAA2F0130031057
:100F58008312D20CD10CD00CCF0CFF3E031DAB2F4B
:100F68000130D300530883160313CA07031DBD2F8E
:100F7800BE2FAA2FEB2FEB2F20304A02031CC52FC0
:100F8800C62FE22F003083120313D2000030D100A5
:100F98000030D0000030CF00FC2FFC2FE22F0130B2
:100FA8008312D3000310CF0DD00DD10DD20DD30B6A
:100FB800D62F013083160313CA02E22F83160313B8
:100FC800CA08031DE82FE92FD32FEB2FEB2F490871
:100FD800031DEF2FFC2F83120313CF09D009D1096A
:100FE800D209CF0A0319D00A0319D10A0319D20A60
:020FF8000800EF
:10100000FF1B0A2883137F1883170008840A03191B
:10101000FF0A080008308A000408840A82070034A6
:10102000633469347234693470342D3445346C342B
:1010300066346F34723475346D342034463465341C
:10104000623420343234303431343934003448346A
:101050007A34003430342E343034303400344B346D
:1010600048347A34003430342E3430340034303460
:041070002E340034E6
:10141A004E346134BC340034033401300A128A1564
:10142A00FF220A128A15080064008001840A040651
:10143A000319003404061A2A003424347434493453
:10144A00E83403340034003483120313B000300844
:10145A0080380A128A15FF220A128A1508000130FA
:10146A008312031390000C10831603130C140B172A
:10147A008B170800831203138510000083120313CD
:10148A0005140000831203130510000008008312DC
:10149A00031385140000831203130514000083123A
:1014AA0003130510000008007E088A007F088200E6
:1014BA000A128A1559220A128A158000840A040817
:1014CA007D0603190034FF0A0319FE0A5D2A00008B
:1014DA000000831203138601C030831603138600AB
:1014EA00831203138501F83083160313850006302F
:1014FA009F0007309C000800831203133908AF00CD
:10150A003808AE003708AD003608AC009630BA008D
:10151A003A08B000B1010A128A1535260A128A154C
:10152A00831203132F08B9002E08B8002D08B7003C
:10153A002C08B600A02A0800FD01D901DA01DB0156
:10154A00DC01DD01DE018313A0308400C9300A12F8
:10155A008A1519220A128A15DC30FD000A30FE00AB
:10156A002130FF00D43084000A128A155D220A1243
:10157A008A156430FD000A30FE000D30FF005F302E
:10158A0084000A128A155D220A128A1583010A1238
:10159A008A15A72C83120313AE002E08AC00043060
:1015AA000310AC0CFF3E031DD52A2C080F39AD00E1
:1015BA002D08AF002F0886000616861600000000C8
:1015CA008312031386122E080F39AC002C08AF00C1
:1015DA002F088600061686160000000083120313E1
:1015EA0086120730AD007D30AC00AC0BFA2AAD0B89
:1015FA00FA2A080083120313AE002E08AC00043046
:10160A000310AC0CFF3E031D052B2C080F39AD004F
:10161A002D08AF002F08860006128616000000006B
:10162A008312031386122E080F39AC002C08AF0060
:10163A002F08860006128616000000008312031384
:10164A0086120730AD007D30AC00AC0B2A2BAD0BF7
:10165A002A2B080083120313B1002D08B301B30724
:10166A002C08B201B2073108B0003008B400552B7B
:10167A003308FF00320884000A128A1500200A1271
:10168A008A15B000340884003008831380000130C2
:10169A00B2070318B30A0130B0003008B407552B5B
:1016AA000130AE020030031CAF03AF02FF302F0639
:1016BA00031D612BFF302E06031D642B652B3D2B6A
:1016CA00662B080083120313CF004F08CD004D0884
:1016DA00CE00CA1F712B722B892B2D30CD004F08DB
:1016EA0084004D08831380000130CD004D08CF07D8
:1016FA00C709C809C909CA09C70A0319C80A0319BF
:10170A00C90A0319CA0A892B4A08BD004908BC003C
:10171A004808BB004708BA004C08BF01BF074B087E
:10172A00BE01BE074F080A128A15C2260A128A1576
:10173A009E2B080083120313B6000F30B100310844
:10174A00B700B82B831203133708AF3E8400831304
:10175A0000080A128A15CF220A128A15013083124A
:10176A000313B702B82B3608B100B201B109B209A6
:10177A00B10A0319B20A31080F3EB300320803183E
:10178A00013E003EB4003408803AB500803035028C
:10179A00031DD12B37083302031CD42BD52BA72BBF
:1017AA00D62B0800710870040319DC2BDD2B122CD0
:1017BA00F501F50AEC2B01300310F00DF10DFF3E97
:1017CA00031DE12B0130F4007408F507EC2BF11F1F
:1017DA00EF2BF02BE02BF22BF22B71087302031D77
:1017EA00F82B70087202031CFB2BFC2B032C7008CD
:1017FA00F2027108031CF303F302032C01300310F5
:10180A00F10CF00CFF3E031D042C0130F502031D00
:10181A000F2C102CF22B122C122C7308F101F10749
:10182A007208F001F007192C080083120313DE0175
:10183A0005305E02031C222C232C252C562C562CF8
:10184A00FD01FD0A282C5E08A03E840083130008CF
:10185A007D050319312C322C382C0A128A154C2298
:10186A000A128A153E2C0A128A153F220A128A1572
:10187A003E2C7D0883120313AC002C07AD002D0803
:10188A00FD00FD08031D4A2C4B2C282C4C2C013042
:10189A00AC002C08DE0705305E02031C552C562CC2
:1018AA00252C0515000083120313051100000800FA
:1018BA000030FC000030FB000030FA000030F90074
:1018CA00662C701C692C6A2C822C7408F90775081E
:1018DA0003110318013E0319732CFA077608031142
:1018EA000318013E03197A2CFB0777080311031822
:1018FA00013E0319812CFC07822C0130F8000310E9
:10190A00F40DF50DF60DF70DF80B842C01300310CC
:10191A00F30CF20CF10CF00CFF3E031D8C2C730837
:10192A00720471047004031D9B2C9C2C662C9D2C44
:10193A007C08F3007B08F2007A08F1007908F000CD
:10194A00A62C0800000000000A128A156C220A124E
:10195A008A150A128A15BD250A128A150A128A15CB
:10196A0034220A128A150000000000308312031381
:10197A00E2000F30E1004230E0004030DF005D1449
:10198A0000000000C82C00000000831203135D1C35
:10199A00CF2CD02CDB2C000000000A128A11152053
:1019AA000A128A15831203135D10DB2CDD1CDE2C50
:1019BA00DF2CEA2C000000000A128A118F260A1274
:1019CA008A1583120313DD10EA2C00000000C82CCC
:1019DA00C82C0A128A111228831203132F082E0404
:1019EA002D042C040319FA2CFB2C442DB501B50A3D
:1019FA000C2D0130B4000310AC0DAD0DAE0DAF0DC2
:101A0A00B40B002D0130B4003408B5070C2DAF1FFC
:101A1A000F2D102DFE2C122D122D2F083302031D0F
:101A2A00202D2E083202031D202D2D083102031D00
:101A3A00202D2C083002031C232D242D332D2C0895
:101A4A00B0022D08031C2D0FB1022E08031C2E0F05
:101A5A00B2022F08031C2F0FB302332D01300310DB
:101A6A00AF0CAE0CAD0CAC0CFF3E031D342D013097
:101A7A00B502031D412D422D122D442D442D33084C
:101A8A00AF003208AE003108AD003008AC004D2D71
:101A9A000800003083120313B8000030B70000308A
:101AAA00B6000030B5002F082E042D042C040319AB
:101ABA005F2D602DB32DB901B90A712D0130B40023
:101ACA000310AC0DAD0DAE0DAF0DB40B652D01308D
:101ADA00B4003408B907712DAF1F742D752D632D0D
:101AEA00772D772D0130B4000310B50DB60DB70D63
:101AFA00B80DB40B792D2F083302031D8E2D2E0835
:101B0A003202031D8E2D2D083102031D8E2D2C0845
:101B1A003002031C912D922DA22D2C08B0022D0803
:101B2A00031C2D0FB1022E08031C2E0FB2022F0820
:101B3A00031C2F0FB3023514A22D01300310AF0C72
:101B4A00AE0CAD0CAC0CFF3E031DA32D0130B90247
:101B5A00031DB02DB12D772DB32DB32D3808AF004D
:101B6A003708AE003608AD003508AC00BC2D0800B9
:101B7A0000000000413083120313B100EE30B000C0
:101B8A00B00BC52DB10BC52D0000831203138612AD
:101B9A000612B20103303202031CD42DD52DD72DE3
:101BAA00F42DF42D033086008616000000008312FF
:101BBA00031386120730B1007D30B000B00BE32D5D
:101BCA00B10BE32D013083120313B0003008B207C2
:101BDA0003303202031CF22DF32DD72DF42D0230DF
:101BEA00860086160000000083120313861207304F
:101BFA00B1007D30B000B00B002EB10B002E0130C9
:101C0A000A128A15FF220A128A1507308312031351
:101C1A00B1007D30B000B00B102EB10B102E0E307B
:101C2A000A128A15FF220A128A1507308312031331
:101C3A00B1007D30B000B00B202EB10B202E043045
:101C4A000A128A15FF220A128A1507308312031311
:101C5A00B1007D30B000B00B302EB10B302E080031
:101C6A00831203133008031D3B2E442E2F082E0423
:101C7A002D042C04031D422E432E5D2E442E0030CB
:101C8A00AF000030AE000030AD000030AC00C12E15
:101C9A00C12E5D2E0130B2003208B00701300310A8
:101CAA00AF0CAE0CAD0CAC0CFF3E031D542E5D2EDA
:101CBA00FE302F05031D622E632E4F2E802E802E9E
:101CCA000130B2003208B0070130AC070030031807
:101CDA000130AD07003003180130AE070030031899
:101CEA000130AF0701300310AF0CAE0CAD0CAC0CD9
:101CFA00FF3E031D782EFF302F05031D852E862EED
:101D0A00652E942E942E0130B0020130B2000310D9
:101D1A00AC0DAD0DAE0DAF0DB20B8C2E942EAE1FC9
:101D2A00972E982E882E30189B2E9C2EA42EFF308C
:101D3A00AC05FF30AD057F30AE05FF30AF050310AF
:101D4A00B00C3008B200B301B401B5011830031069
:101D5A00B20DB30DB40DB50DFF3E031DAC2E320806
:101D6A00AC043308AD043408AE043508AF043108B6
:101D7A00031DC02EC12EAF17080083120313C6001D
:101D8A003D08C4003C08C3003B08C2003A08C10031
:101D9A00CE2E3E08AC003F08AD000030AD1BFF3030
:101DAA00AE00AF004408B3004308B2004208B100D5
:101DBA004108B0000A128A154E250A128A158312A2
:101DCA0003132F08C4002E08C3002D08C2002C08D4
:101DDA00C1000130C0004008C60744084304420459
:101DEA004104031DF92EFA2ECE2EFB2E460884003E
:101DFA00831380010130C602022F3E08AC003F085F
:101E0A00AD000030AD1BFF30AE00AF003D08B3009F
:101E1A003C08B2003B08B1003A08B0000A128A1521
:101E2A00F1240A128A15831203132C08C0004008F1
:101E3A00C5003E08AC003F08AD000030AD1BFF30C6
:101E4A00AE00AF003D08B3003C08B2003B08B10049
:101E5A003A08B0000A128A154E250A128A15831208
:101E6A0003132F08BD002E08BC002D08BB002C0848
:101E7A00BA000A304502031C432F442F482F07306B
:101E8A00C0004008C5073030C0004008C5074508F3
:101E9A00C000460884004008831380000130C6024F
:101EAA003D083C043B043A04031D5C2F5D2F022FBE
:101EBA005E2F0800831603134E0883120313B9001A
:101ECA00831603134D0883120313B80083160313F2
:101EDA004C0883120313B700831603134B088312AB
:101EEA000313B6000A128A1581220A128A1583126E
:101EFA0003133908C2003808C1003708C000360881
:101F0A00BF004130BE00BE30BD00E330BC002F3000
:101F1A00BB000A128A1179250A128A158312031341
:101F2A003E08D2003D08D1003C08D0003B08CF0053
:101F3A000A128A1148270A128A15831203135208B1
:101F4A0083160313A800831203135108831603137D
:101F5A00A70083120313500883160313A6008312E3
:101F6A0003134F0883160313A5002508CF004F0853
:101F7A00A0002508CF002608D0002708D10028088D
:101F8A00D20008300310D20CD10CD00CCF0CFF3E7B
:101F9A00031DC72F4F08D3005308A1002508CF00FF
:101FAA002608D0002708D1002808D20010300310D4
:101FBA00D20CD10CD00CCF0CFF3E031DDC2F4F08E6
:101FCA00D3005308A2002508CF002608D00027080E
:101FDA00D1002808D20018300310D20CD10CD00C32
:101FEA00CF0CFF3E031DF12F4F08D3005308A30067
:061FFA00A401A40A080086
:02400E007AFF37
:00000001FF
